:10000000200B0020F1000000ED000000ED000000DA
:1000100000000000000000000000000000000000E0
:10002000000000000000000000000000ED000000E3
:100030000000000000000000ED000000ED000000E6
:10004000ED000000ED000000ED000000ED000000FC
:10005000ED000000ED000000ED00000000000000D9
:10006000ED000000ED000000ED00000000000000C9
:1000700000000000ED000000B9130000C5120000F0
:100080000000000000000000ED00000010B5064C6C
:100090002378002B07D1054B002B02D0044800E049
:1000A00000BF0123237010BD2000002000000000CD
:1000B00068270000084B10B5002B03D007490848FB
:1000C00000E000BF07480368002B00D110BD064BBD
:1000D000002BFBD09847F9E7000000002400002027
:1000E000682700006827000000000000FEE700000D
:1000F0001D481E4970B5884202D000231C4C03E005
:100100001C4B1D4A002106E0CA18A242F8D2C5586D
:1001100004331560F8E7934201D202C3FBE7FF21E5
:100120000220164B164A8B4393603022154B5862BF
:10013000154B997B9143103A11439973997B143A6B
:100140009143043A1143997303219A7B8A430243F2
:100150009A730E4A7D3153680B4353600C4B98479A
:100160000C4B9847FEE7C0466827000000000020BF
:1001700020000020200000202007002000000000B8
:1001800000ED00E0FC7000410048004100400041EB
:1001900085200000A11900000300F0B538331B785A
:1001A00087B0049303000500002639331F780368E5
:1001B0005B7C05932B68B1B21B7CF4B2D800414341
:1001C000686B89B241183A1903940091094CD2B274
:1001D00000212800A047039C049B0134E4B2A34201
:1001E00005D90136BB19059ADBB29A42E2D807B0AD
:1001F000F0BDC046B1100000020010B503683832EF
:100200001B7C1278406B5A430021D200014B984767
:1002100010BDC046D120000010B50400024B984725
:100220002000024B984710BD99010000F510000016
:10023000030010B539331970036B1B68984710BD64
:10024000030010B57E331B780400002B01D0034B54
:10025000984700212000024B984710BDF90100008B
:100260003102000070B504000F4B9847230039336A
:100270001D78013B1B78ED182368EDB25B7CAB4227
:1002800004D82000094B984700200CE023007E335F
:100290001B78002B02D02000054B98472000290036
:1002A000044B9847012070BD99010000F510000033
:1002B000F90100003102000010B5044B040098471A
:1002C0002000034B98470028FAD110BD41020000DE
:1002D0006502000008230370004870473C000020BE
:1002E0007FB50E00009309491300094D094A040027
:1002F000A8470F256D442800074B98472A7801002E
:1003000000962000054B064CA0477FBDF111000070
:1003100071120000FD0F0000D5020000E509000089
:10032000290E0000411808784B780002C01880B2EE
:10033000704710B54418E4B2012B09D08418E4B218
:10034000002B05D0821AD4B2022B01D0401AC4B2BD
:10035000200010BD30B5851AECB2012B09D045182C
:10036000ECB2002B05D0411ACCB2022B01D082187E
:10037000D4B2200030BD00207047000070B50B786B
:100380000D0003704B78040043708B788370CB783A
:10039000C3700B7903714B7943718B798371CB797E
:1003A000C3710B7A03724B7A43728B7A8372CB7A66
:1003B000C3720B7B03734B7B43738B7B8373CB7B4E
:1003C000C3730B7C074E037411212800B04713211F
:1003D00060822800B0471521A0822800B047E08243
:1003E00070BDC0462503000070B5867A0468721897
:1003F0002378D2B23341072A01D8DBB20AE0651C68
:10040000056065780824A41BE4B2A540083A2B4394
:10041000DBB2D2B28272012088400138184070BD30
:1004200070B50400002350340165A3720300050079
:100430006433094E19782000B0472B0020726533D1
:1004400019782000B0477D3560722B7823735A42AB
:100450005341637370BDC046E903000010B50C0042
:10046000044B98470123013CE4B2A340C01A40B2B8
:1004700010BDC046E90300000300F0B504000F0002
:100480008DB00B9250339A790292DB790593250057
:1004900050352B7A029A9B1ADBB20393039A3B1CCA
:1004A000974201D96B461B7BDBB208936B792879A5
:1004B00008260A936B469E571B7D31005BB206935C
:1004C000AB7B069A0796194E0493B047049B09909C
:1004D000069A07990A98164EB0470B9B0200002B0C
:1004E00001D0297B03E0EB7A002B0AD1697B230042
:1004F0007D331970049B099900932000089B0D4DD2
:10050000A847039B9F4208D3FB1ADFB2059B013328
:10051000DBB2059300230293B9E7029B5034FB182A
:10052000A3716B461B7EE3710DB0F0BD5503000057
:1005300033030000430900000300F0B504008BB052
:1005400050330393524B9847230059331B78514D36
:100550005BB207932300663319780398A8472300FA
:100560000890673319780398A847230068331978EF
:1005700006000398A847039B09901B7A5BB204937B
:10058000002B00DC81E06B461B7F089905939E19C8
:10059000039B76429B7B76B20693039B32001879CD
:1005A0003D4D069BA847039B320018710899050032
:1005B00007003A4E5879069BB047039B02005871DA
:1005C000069B0100032B2CD8180001F0DBFB02096D
:1005D0001220049B0598EF188118FBB2C9B222E0E3
:1005E000059B0498ED1A013711180135FBB2C9B209
:1005F0000BE00122049B0598D51A7D19BF18121A29
:100600008A180131FBB2C9B2D2B2EDB20BE0049A42
:10061000059B8A1A5F1901320131FBB2C9B2D2B20D
:1006200001E001002B000091200029001C4DA8478B
:1006300000282AD02300002250339A71DA71230057
:1006400062331978174D0398A847230063330700D6
:1006500019780398A8470600002239002000124D9F
:10066000A847310020000122A847012103980D4B23
:1006700098470028F0D12300072250339A56079953
:100680008A42DCDB1B7B7D34237009980BB0F0BD04
:10069000210400005D040000550300003303000046
:1006A000B1090000E903000079040000826C1732F0
:1006B000FF2910D8602901D9743002E0402902D9FD
:1006C00072300388D2185378002B13D010788842E8
:1006D000F8D1901C0FE0763000881018037842782B
:1006E0001B02134306D0994201D1033003E0837803
:1006F000C018F3E718007047F8B51F0003005E3319
:10070000040018780E001500032815D8E36C01F0DA
:1007100039FB02060A0F200098472D1806E020003A
:100720009847361A07E0200098472D1AEDB203E0EB
:10073000200098473618F6B2230054331E705D70BF
:1007400039002000044B9847011E03D02000034BC2
:100750009847C0B2F8BDC046AD060000390500009C
:10076000F7B50193194B06000C00150098470023BC
:100770000093019B3000197873689847144A031E50
:10078000934221D0019A01320192124A9042F0D054
:100790002A0021003000104FB84732005E320300BB
:1007A000107803280CD801F0EDFA02040609E418C9
:1007B00002E0ED1803E0E41AE4B201E0ED1AEDB254
:1007C000009AD318DBB2D3E70098FEBD750E000087
:1007D000FFFF0000FEFF0000F906000010B5024C0C
:1007E0004460024CA04710BD610E0000610700008C
:1007F000836C70B5002B2BD003000026050001246C
:1008000002006D339E5779352E701C577A32147062
:100810000B331B78002B1BD0012B0CD103006F3343
:100820001B785BB29E4200DA2B707023C3569C4249
:100830000EDD13700CE003006C216A331B78415607
:100840005BB25B189E4200DA2B708C4200DD1170A7
:1008500070BD0000014BC3647047C04677030000C1
:1008600010B5836C04008B4206D08164034B60306A
:1008700098472000024B984710BDC0467D030000FA
:10088000F107000073B5060006AC24783A36012B58
:100890000ED135788D4253D9050039352D78ED00CC
:1008A000521B05003B352D78D2B2954248D944E021
:1008B000022C03D10131C91AC9B204E0032C02D1C0
:1008C0000132D21AD2B201252C40050039352D78DB
:1008D0003678ED00521B05003B35D2B22D78002C46
:1008E00015D1AA422CD2CB18DBB2994205D9B1421C
:1008F00002D2731EDBB202E021008E4220D9002B0F
:100900001ED0351C9E4200D91D1C6B1A14E0B1424A
:1009100016D29B18DBB29A4205D9AA4202D26B1EAC
:10092000DBB202E0002295420AD9002B08D02E1C2F
:100930009D4200D91E1CB31ADBB20094C46AA047C2
:1009400073BD37B506AC2578002B03D0046B00953A
:100950006468A04737BD0000F0B51500013285B0CE
:10096000D2B21F00CB180092DBB22A00074E0390D0
:100970000C00B047002807D00023210000932A0074
:100980003B000398024CA04705B0F0BDB109000040
:10099000430900008A4206D20121834206D89342CD
:1009A0009B41594202E08342F9D800210800704778
:1009B000F8B50E00010004001F00443106AB4330BF
:1009C0001B7809780078064DA847002807D0230037
:1009D00041344233197820783B003200A847F8BDF3
:1009E00095090000F7B508AC247807260194012486
:1009F00005001640B4407D3500912F78E4B2002503
:100A0000012F03D82500012F00D100240727BA4366
:100A100011000268127C4A4300995118426B511828
:100A2000019A002A09D10A78013B2A436240DBB2CD
:100A30000A700131002BF6D120E03A22944684441A
:100A40007D300A7801362A436240013B0A703E40FD
:100A5000DBB2002E0AD16246127889180278012A88
:100A600009D80125AA4207D02C0005E06D006400DA
:100A7000EDB2E4B200E00124002BE2D1F7BD10B5E5
:100A80000822845E0A21425E03000020A24215DD96
:100A900099899A88D8898918DA8889B2821892B295
:100AA00010B29981D881002805DD1888091899812C
:100AB0005988521ADA81012001341C8110BD037E4D
:100AC0000131C9B299429B41194008007047013970
:100AD000007EC9B2814201D30138C1B2080070471B
:100AE0001823534370B5C4182300050030330E009B
:100AF0001978E36A280098478300EB1802229B5E6E
:100B00000100B34203D1230030331870F1E770BD08
:100B1000F8B51823020059431C325418217D0600F1
:100B20008B00C31802229D5E0027DF5F2369984770
:100B30008300F3180222995E00229B5E4A1BDB1B96
:100B40009BB292B2207516B218B26680618125817F
:100B5000A781002805DB0123238000230500E38112
:100B600007E05D420121012349429A1A21802DB2FA
:100B7000E2813100044B98473100A080034B2800EC
:100B80009847E180F8BDC046AD1E00007920000006
:100B9000037E10B5052B05D89C0004190133218074
:100BA0006280037610BD0000F7B5574B0091436497
:100BB000564B0400C3620222835E0200303201926F
:100BC00000221D00019906300A70877C0132BA426A
:100BD0000FD20026815F0E1C994200DA1E1C33B230
:100BE000A94202DA019D2A700D000132D2B204300E
:100BF000EDE75B1B1BB26383002B00D182E0260074
:100C0000019B48361B780122337029002000404F99
:100C1000B847290000222000B84701236376019BD2
:100C20001A78337892009B00125F1B5F9A4202D0C1
:100C30000023637605E0638B013B1BB26383002BCB
:100C400060D0270000212000324E1A23E55EB04715
:100C500001212000B047637E1C37002B05D03800EF
:100C60002D4EB04720003430B0473C23E25E002ACE
:100C700031DB009B40331B789A422CDA2823E05E5C
:100C8000A31C3E215B5E984211DA002B23DB009906
:100C90003F310E78B0421EDA011C002800DA002134
:100CA00009B29E4200DC33B2C9B25B1A0EE00028E2
:100CB00011DB00993F3109788B420CDADE43F617DD
:100CC0003040814200DC08B2D9B2431ADBB2D2B262
:100CD0000098124EB04738000F4EB047011E03D1A6
:100CE00020000C4B9847F6E720003430B04700282E
:100CF00004D101212000074B9847F5E7013D2DB2B3
:100D0000002DB2DCF7BDC046BF0A0000CF0A0000CC
:100D1000E10A0000110B00007F0A000059090000E1
:100D200010B50100014B0248984710BDA90B000007
:100D300094040020F7B50600100008AA0024125FF2
:100D400009AC0025645F0A4D01940AAC0027E75FF7
:100D5000084C218001216080217620001900A847DD
:100D60003A0001992000A8473000034B9847F7BD8F
:100D7000910B000094040020210D000003000200EC
:100D800070B538331B783B32D900117001680C7C88
:100D9000221C1F2C00D91F220400D2B23A34D200E8
:100DA0002270020039321578EA00D2B2A2704C7C6F
:100DB0005E19A64201DD631BDBB20400DB003D349B
:100DC0002270D31802003E3213700300F0223F332A
:100DD0001A708A8AF02A00D81A70CB8A40300370C1
:100DE00070BD000010B50400094B98472300002295
:100DF00041331A7022003A321278033B1A712200F2
:100E00003D32127844345A711B78237010BDC046AD
:100E10007D0D000013B504AC24780094014CA0476C
:100E200013BDC0468508000070B50400E3622300CE
:100E300000253833A56461631A7022005D700123B8
:100E400004987D3213705370206303682000984724
:100E50002000024B5E349847257070BD5508000095
:100E6000002902D088B20A2900D101487047C04643
:100E7000FFFF000000230430C377704710B50A005D
:100E8000046900232021A04710BD10B51300046998
:100E90000A001721A04710BD07B56B46DA1D117077
:100EA000014B012198470EBD8B0E0000143970B51F
:100EB0000400081E0C2842D800F064FF14414107CA
:100EC0002432414141414141220001201D499A18EB
:100ED000934232D01C781B4D8C622C7E0442FCD095
:100EE0000133F5E70125236820005A784921164E81
:100EF000B047236840211A7B20002A40B0471CE0FD
:100F00004A2117E0236820001A7849210E4B9847A0
:100F1000236865699A782C2100232000A8470CE0FB
:100F200023682C21DA78200000236569A84749212D
:100F300023685A782000044B9847012000E00020E5
:100F400070BDC046000800423912000010B50A000A
:100F5000C46800231521A04710BD10B50A00C4685D
:100F600000231621A04710BD10B51300C4680A0065
:100F70001721A04710BD002310B51A00C46818211E
:100F8000A04710BD002310B51A00C4681921A0475E
:100F900010BD000073B505000C002178172916D08C
:100FA00009D8152925D36B4662782800DA71EE68D6
:100FB0000023B0471BE0192912D9FE2919D16B462D
:100FC00062782921DA7128000A4B98470FE06B46B6
:100FD000DA1D6378012113702800074B984706E05B
:100FE000002328001A00EE680134B047D5E7023428
:100FF000D3E773BD39120000690F0000F7B5019304
:101000000B00143B04000E0015000020052B19D81E
:10101000180000F0B7FE1103030D111100210A4B57
:101020002000984729002000084B9847012009E03C
:1010300001212000044B98472769019B2A003100B9
:101040002000B847FEBDC0467D0E0000990E00008E
:1010500001608B7C83777047002370B51A002821CC
:1010600045690400A8470023E5681A001421200000
:10107000A8470E4D200001224B21A84723682000DD
:101080001A792921A847200000224B21A84723686C
:1010900020001A792921A847200001224B21A847C6
:1010A000236829215A792000A84770BD3912000011
:1010B00013B56C462371049B6171A271009384681F
:1010C0006B4601220F21A04716BD002310B51A0060
:1010D00084680921A04710BD002310B51A00846858
:1010E0000A21A04710BD10B50A00846800230B2117
:1010F000A04710BD002310B51A0084681021A04736
:1011000010BD0000F7B50B39040015001E00081EC5
:10111000042856D800F036FE03550B1B2B002A4B33
:101120002A49002A00D02A49200098471DE0264B72
:10113000002A05D127492000984723689B7C04E0BA
:101140002549200098472368DB7CA3770DE0234BDB
:10115000200098478121224B200098472900200039
:10116000204B98472000204B984701202AE01B4B3A
:10117000200098477179A37FC900C918CBB2184FD6
:10118000402120000193B8471021019B20001B093A
:101190001943B8470F21019B20001940114FB84750
:1011A000B023B17920001943B8473179013DC90016
:1011B000C9B2326820000D4BEDB29847002DF4D132
:1011C000D0E70020FEBDC046950F0000A02600001D
:1011D000A5260000C426000000270000770F0000AD
:1011E0004D0F00005B0F0000850F0000690F00002D
:1011F00070B50B4E04000D00B04700280ED1092D2C
:1012000008D00A2D0BD12000064B98470649200034
:10121000064B02E020000649064B9847012070BDAE
:101220000511000059100000CB260000950F0000AA
:10123000AC2600005110000010B500234469A047FF
:1012400010BD0020704700000023084AC377826069
:10125000C26002614261C21C0360D377021DD37772
:10126000421CFF330630D377C37770474312000028
:10127000F8B504000F0016001D00054B9847069BAB
:10128000A760E660256163612000024B9847F8BDC6
:1012900049120000CB100000492906D04A290FD17D
:1012A000C0238021DB05490203E0C0238021DB0548
:1012B000C900002A01D0996100E05961012000E0D5
:1012C0000020704770B5324A324B1188002911D086
:1012D00031490978002905D030485C8B01686118D4
:1012E000016007E0598B2E482E4C09B2018020681E
:1012F000091821601188013189B2118011882029D3
:1013000042D90020244910800A78D2B2824216D0F5
:1013100018705A7E52B2002AFBDB01201D4A106170
:101320005A7E52B2002AFBDB02201A4A10705A7E03
:1013300052B2002AFBDB0222164B1A731FE0194C33
:101340001948256805601548184D06682E6022600A
:1013500001240260164804701A705A7E52B2002AA4
:10136000FBDB14480B4A10615A7E52B2002AFBDBA9
:101370000220084A10705A7E52B2002AFBDB01227A
:101380000B7853400B7001E002221A7370BDC04607
:10139000480400200020004210000020EC0400203F
:1013A00008050020F0040020E80400201C070020AD
:1013B0004A04002003190000012270B50B4B0C4DAC
:1013C0009A730C4A0C4B11681B68CB18FA211360F6
:1013D0000A4B890018680A4B98470A4A2C68136818
:1013E000041901332C60136070BDC046001C00421C
:1013F0004C040020640400206804002074040020D1
:10140000AD1E000050040020F7B50026C317C51814
:10141000114C00915D40571C7B1E0193009BB34211
:1014200003D12E227B1E1A7010E0210028000B4BE6
:1014300098477B1E3030187021002800084B9847D1
:1014400020000D00074B0A21984784B2013601376E
:10145000062EE1D1F7BDC04610270000AD1E0000EA
:1014600079200000991D0000F0B585B003930700B6
:10147000019102920A9C1E4E20231E4D00280EDD73
:10148000092804DD0A21B0473030207000E02370C5
:101490000A213800A84730316170642301E02370CD
:1014A0006370A3702023E3701A33A37163720A215F
:1014B0000198B047303020710A210198A847303197
:1014C000617102980A21B0473030E0710A21029818
:1014D000A8473031217203980A21B0473030A072FA
:1014E0000A210398A8473031E17205B0F0BDC0462B
:1014F000AD1E00007920000000220120130030B54D
:1015000007494042940065589D4200D963580D59DF
:10151000854200D208590132642AF3D1181A30BD2D
:101520008C0500200123044A10689900013388507B
:10153000642BF9D17047C0468C050020802300221F
:10154000F0B56A4DDB036B61694B6A4C1A708432EB
:101550005A70694822680168127809781202521894
:10156000D2081A850A221E009A7087B03532DA70C6
:10157000029503940490737E5BB2002BFBDB5F4A01
:101580005B4B1A61737E5BB2002BFBDB1122584B65
:101590009A80737E5BB2002BFBDB0222544B1A70E5
:1015A000737E5BB2002BFBDB0122514BDA75737E3D
:1015B0005BB2002BFBDB20240025022201213273C9
:1015C000337E4B4F0B42FBD07B8B013C1BB2E4B212
:1015D000ED18002CF3D14A484A4968434A4B9847D2
:1015E0004A4B4B491860FA20C0006843464B984765
:1015F000484B4949186042483961019042482025CA
:10160000844622000227012005913773317E384C31
:101610000142FBD0618B013D09B2EDB25218002DA1
:10162000F3D1FA20C0001F685043634638499847F9
:101630003A4BC71B1F600123202723612800022289
:101640001C003273337E2342FCD0294B013F5B8B5D
:10165000FFB21BB2C018002FF3D12C4B2A4D1C68CF
:10166000019B284943431800A8472D4B041B2B4AD4
:101670001C60106812682B4901921C68A84735301D
:1016800060436421A847BC21040089000198A84751
:10169000254B241A993C1C608023029ADB0393613A
:1016A000134B1F70039B049A1B6812681B781278F7
:1016B0001B029B180E4ADB081385737E5BB2002B5E
:1016C000FBDB0B4B059A1A61737E5BB2002BFBDBD5
:1016D000737E5BB2002BFBDB0222054B1A70737E1C
:1016E0005BB2002BFBDB07B0F0BDC04600440041FD
:1016F000002000420C000020080000200202000030
:101700001027000099990100AD1E00004004002040
:101710006D1700005C040020031900007004002015
:10172000900400208D2000008804002070B5114C2A
:1017300011492000114B9847114B124D1B68102284
:1017400019212000A847104B20221B680A212000E5
:10175000A8470E4B30221B680A212000A8470C4BDB
:1017600040220F211B682000A8472000094B984702
:1017700070BDC0460C050020E0200000610800009C
:1017800014000020DD0700001800002004000020E5
:101790001C00002019020000554B564A70B5938278
:1017A0000223D1681942FCD0534B544999605978AF
:1017B000C909FCD152485049486059784E48C90976
:1017C000FBD150491E2441608421C90141804E480B
:1017D0004168A1431A3C214341601020D468454927
:1017E0000442FBD0062088844848C8621021D06893
:1017F0000842FCD0464A5A6059783F4AC909FBD191
:101800004449518044495180444991604449516060
:101810005A78D209FCD14349374B43485980434B4E
:10182000434999601A6111232221424A1370424AA6
:101830001370424A103B1370414A1170414A1D39DE
:101840001370414A1370414A1370414A1370414A60
:101850001170414A7F311370404A1370404A136A35
:101860000B4313620222C1692F4B1142FBD13D4A47
:1018700002211A6001221A73802292025A60DC69E6
:10188000294802220C42FAD1016811430160D9694A
:101890001142FCD10122344B5A7305321A80DA7B93
:1018A00052B2002AFBDB314C314A32492000324B24
:1018B000324DA8472000324B984700212000314B81
:1018C0009847626B304B20001A60304B9847304B82
:1018D0009847304B984780222F4B12021A60802283
:1018E000D2011A6062B602222C4B1A7370BDC04638
:1018F0002E06000000080040000C0040018000009F
:10190000010501000205010000400041B905082061
:1019100000070100124100000E4000000304000017
:101920000307030013430000000800420044004185
:1019300000C441003144004132440041334400417D
:101940003744004142440041434400414444004183
:1019500045440041464400414E4400414F4400414B
:10196000000400400C003000001C00420C05002068
:10197000AD0E00009826000099120000E102000060
:10198000D9100000E7100000E4040020B9020000B4
:101990002D1700003D15000000E100E0002000428E
:1019A000F0B5C44B89B09847C34B1A78D2B20592B0
:1019B000002AFAD0C14BC24E1C68C2492000B04771
:1019C000C14BC24D18603C212000A847C04B2000ED
:1019D00019603C21B0473C21A847BE4B200019604C
:1019E000E1210901B0471821A847BB4BBB4D196045
:1019F000BB4BBC491B68BC4C0693BC4B1868BC4B2A
:101A000068431F68B047C71BFA20BA4BC0001E6866
:101A1000069B27605843B849B84B9847B84B861B7C
:101A2000B84F1868B84B3E60361A1E601A68002A14
:101A300002DA1A6852421A601B68AB4203DD72B6C2
:101A4000B24B984762B623681A00643201DAB133A8
:101A500023603D6826680A21A84C2800A0470A2177
:101A60000700974B300098474743A94BA9491F608F
:101A7000A94B0A881E60A94BA9481D60A94B1F608D
:101A8000531C9BB292000B801550642B01D900238C
:101A90000B80A54D2B78002B03D0A44B9847002337
:101AA0002B70A34B98470022A24BA34D1860824B8A
:101AB00028001A708C4B1F68FB17FF185F409F4B64
:101AC000984728009E4B9F4998478E4B9E4E18681A
:101AD0009E4B984204D90A21A0473200022101E01E
:101AE000320001219A4B9847974C9A4E23001A22B4
:101AF00000212800B047380022000121944FB84748
:101B00002300280026220021B047864B804D1B6809
:101B100006970796002B00DA5B422B602868684F17
:101B20006421B847012600232860884A904205DDD9
:101B30000A210136B847F6B2059BF6E7002B00D024
:101B4000286031002200069B9847230032220021A2
:101B5000079D7948A847E1217F4B594E1868090134
:101B6000B0470125794B984204DD0A210135B04781
:101B7000EDB2F7E729002200069B984723002622B2
:101B80003D21079D6C48A847B421744B4C4E186802
:101B90004900B04701256D4B984204DD0A2101350B
:101BA000B047EDB2F7E722002900694FB847624D10
:101BB0002300684E32223D212800B0475D4B2200B1
:101BC00018680421B84723001A223D212800B04795
:101BD000634C3F4B3F4A40493B4800941B681268A6
:101BE000096800685F4FB84723000E2217212800BC
:101BF000B0475D492800524B98475C4C56231A2247
:101C00002D212800A047412326222D212800A0476E
:101C1000572332222D212800A047572332226A2140
:101C20002800A0476823322277212800A0474123BB
:101C300026226D212800A04768232622772128002C
:101C4000A0476D231A2219002800A04756231A2204
:101C500077212800A047244B454F1A68032302939D
:101C6000002A0CDA08241B19009307222300042100
:101C700001942800B8472300072221000AE07823B6
:101C80000B22019300927C21043A2800B8470823D4
:101C9000072271212800374CA047374B40221B6890
:101CA00019212800B047354B280098470222344BB1
:101CB0001A7379E6991700004A04002050040020A6
:101CC000AD1E000080510100780400207920000042
:101CD0005804002084040020600400201027000025
:101CE0001C0700209999010044040020E80400200A
:101CF000880400205C0400206D170000991D00007E
:101D000070040020800400203C0400203D150000E9
:101D1000540400207C040020680400208C0400206F
:101D20008C05002074040020000000202515000010
:101D3000F91400006C0400200C050020F9010000DB
:101D400061080000E1250000010500209F860100D8
:101D500009140000DD070000640400204C0400208A
:101D6000F404002069140000E0200000F9060000DF
:101D7000350D000059090000140000201902000070
:101D80000020004202B4714649084900095C49003C
:101D90008E4402BC7047C046002243088B4274D375
:101DA00003098B425FD3030A8B4244D3030B8B425C
:101DB00028D3030C8B420DD3FF22090212BA030C65
:101DC0008B4202D31212090265D0030B8B4219D346
:101DD00000E0090AC30B8B4201D3CB03C01A524166
:101DE000830B8B4201D38B03C01A5241430B8B42AE
:101DF00001D34B03C01A5241030B8B4201D30B0397
:101E0000C01A5241C30A8B4201D3CB02C01A5241BD
:101E1000830A8B4201D38B02C01A5241430A8B4280
:101E200001D34B02C01A5241030A8B4201D30B0269
:101E3000C01A5241CDD2C3098B4201D3CB01C01A83
:101E4000524183098B4201D38B01C01A524143098D
:101E50008B4201D34B01C01A524103098B4201D37B
:101E60000B01C01A5241C3088B4201D3CB00C01AE8
:101E7000524183088B4201D38B00C01A5241430860
:101E80008B4201D34B00C01A5241411A00D2014685
:101E9000524110467047FFE701B5002000F0F0F80E
:101EA00002BDC0460029F7D076E7704703460B43D2
:101EB0007FD4002243088B4274D303098B425FD343
:101EC000030A8B4244D3030B8B4228D3030C8B426F
:101ED0000DD3FF22090212BA030C8B4202D3121255
:101EE000090265D0030B8B4219D300E0090AC30B2A
:101EF0008B4201D3CB03C01A5241830B8B4201D3D7
:101F00008B03C01A5241430B8B4201D34B03C01ABF
:101F10005241030B8B4201D30B03C01A5241C30A37
:101F20008B4201D3CB02C01A5241830A8B4201D3A8
:101F30008B02C01A5241430A8B4201D34B02C01A92
:101F40005241030A8B4201D30B02C01A5241CDD237
:101F5000C3098B4201D3CB01C01A524183098B4282
:101F600001D38B01C01A524143098B4201D34B016B
:101F7000C01A524103098B4201D30B01C01A5241CE
:101F8000C3088B4201D3CB00C01A524183088B4255
:101F900001D38B00C01A524143088B4201D34B003E
:101FA000C01A5241411A00D20146524110467047B0
:101FB0005DE0CA0F00D04942031000D340425340B5
:101FC00000229C4603098B422DD3030A8B4212D375
:101FD000FC22890112BA030A8B420CD389019211A7
:101FE0008B4208D3890192118B4204D389013AD0E4
:101FF000921100E08909C3098B4201D3CB01C01AB9
:10200000524183098B4201D38B01C01A52414309CB
:102010008B4201D34B01C01A524103098B4201D3B9
:102020000B01C01A5241C3088B4201D3CB00C01A26
:10203000524183088B4201D38B00C01A5241D9D23E
:1020400043088B4201D34B00C01A5241411A00D2BF
:102050000146634652415B10104601D34042002BBB
:1020600000D54942704763465B1000D3404201B53A
:10207000002000F005F802BD0029F8D016E77047EF
:102080007047C0460E4B70B500251E000D4CE41A7B
:10209000A410A54204D0AB00F35898470135F8E7E7
:1020A00000F052FB084B00251E00084CE41AA41057
:1020B000A54204D0AB00F35898470135F8E770BD4E
:1020C0005427000054270000542700005827000020
:1020D00003008218934202D019700133FAE7704767
:1020E0005F00030204040305050D1000FD0AFD0A4C
:1020F000FD0172037004E8200500EC132107A1859F
:10210000138728220733BD1589252315A78477490E
:10211000988449344C499844C39484499864002471
:102120000FD4755659A44446319312298B002516B5
:10213000AA853CB21426519669399223399269A531
:10214000248C64052614A8855A7192266912474B7F
:1021500029C992629425D116270631BD1303280A96
:10216000D26D3489D29F9200290BD26D144994F418
:102170008B92002A0A55AD5795CAD214012B0A55E5
:10218000955761344861042C0732743389022D0756
:1021900014A41443002E06118513012F0CC474746B
:1021A0004D59292B653500300AA485364AE44F89FC
:1021B000023109A3863689D42F03320DA485364A0D
:1021C0009495B2288BA241330DA485364A9455C408
:1021D0002C931205340BA4857691A5451AB40635C7
:1021E0000DA4851683561BB34C4A1400360DA485E6
:1021F000564A94654BE4942800370CA485168394C2
:102200004559296B02380DA485364A644A94C82979
:102210005100390CA485364AE4946CA544023A076F
:1022200061851361003B09827433399428003C08AE
:1022300095859759D70E3D09459D17838E0D023E12
:102240000995851769B78E003F0CA485364A949589
:102250006A3918014015AA855CC31627D92495A4AC
:102260009254924ADA94A4DA0A4114A984993992D0
:1022700003499CA459988583964669B20D4214A7D8
:102280008519A73009933019A430099330098721A3
:10229000014313A8855A43529C752007722007E218
:1022A00024CC86084415A8851A8398496194266928
:1022B000922669124699326800450FA68518972C18
:1022C00049A368885A6BC310460FA68518972C49F6
:1022D000A368885A8B1B004716A9855A4312854A62
:1022E0009CE4488EA4439CC4519A0D12004814A843
:1022F000851AD31246611446C314466114466132EE
:102300000D4909A385154BD42F034A0BA585575BAF
:10231000D8972899004B12A88519CB9495C224957B
:1023200093340AB362320D4C0AA785196BDC8FC354
:10233000204D14A9851BAAA2499AA4494953D294B5
:1023400034F56549064E15A8851ADAA2455A944413
:1023500095A825AA449994295B024F0FA8855A4352
:102360001626B1CF49980D11005011A685188394F7
:10237000255992255932446971035111C8755A4340
:102380001626B1CF49980DB10E28005210A8851A13
:102390008398F5DB104661564C3601530DA5853701
:1023A000A64D55536D5214005414A9851B0F593175
:1023B0004772244772244772240736005515A885B2
:1023C0001AD31246611446611446611446613644BC
:1023D000005614A98419DB92466956CCD2244EE2E9
:1023E0002407722404571AAD841D8B65C9922CCA28
:1023F00092AC63564D9A93E6A41DC872240B015803
:1024000015AA841AE31267611AE5808EE840948663
:10241000599C8C035914A98419DB9266C52C4D7202
:1024200020477224477260035A0EA88418AF710EB9
:10243000C4ED409C0E075B08D26D144BFF455C0C4D
:10244000C4741459312B66C5AC005D08D26D144AB2
:10245000FF655E0835C55759520B5F06166C1607A7
:10246000600733C4145901610D7585366AB4444957
:10247000944491126211A685176A8B2425599225DE
:102480005992450B00630B7585364B26B6250B001C
:10249000640CA585766265D0BC254300650D758505
:1024A000364BA60D4398250B00660BA485554A169E
:1024B0004D5937056712A66D37C3966449164DF11D
:1024C000908462322400680FA78417728B26D5A2ED
:1024D0002CCAA22C326909A385343920F5246A0A52
:1024E000D26D34A1D22F0A006B0EA78417729354B9
:1024F0004BC231CA4A066C08A38413527F126D0D79
:102500007984194A94294AD4FF49316E0E77841789
:102510008A26D5A22CCAA22C326F0A7585364BE6C4
:102520002D59007013A66D178A24255992255992AA
:10253000254394861B007111A66D3743922559924D
:1025400025599245435A1C720B7485154A22656DB4
:102550000A00730973853453565A00740A938534FC
:1025600051B244DD02751077841792944559944511
:102570005914698A00760E778417CB924559254CF9
:10258000D23803770F798419CA2DD32A9D92B66267
:102590001601780C778417CB9255D24A56397911A7
:1025A000A76C17CB924559254CD2380D9350057A1C
:1025B00009758516B7DE86017B0BD36D5549D42589
:1025C0008BBA057C07D16D131F027D0CD36D155995
:1025D000D42D89BA44007E0726C538920500000034
:1025E000000D0003030304030405060C01FE0A00AA
:1025F0000A0000000000009E2005801B052E068AB0
:10260000228500300ED622962C1411F149128A89A7
:10261000003108D522D621B43F320ED6220E4544D1
:1026200012CA4632D94C68330FD6220E4532541A9C
:102630000E8594090500340DD622A66C448AA89014
:102640000E410D350ED622C621A858150A29130AA7
:10265000003610D622D62844145626249224141369
:1026600001370CD622866D4D2813CA36013811D693
:1026700022962C1411912414119324141301390F50
:10268000D622962C1411B14C8A425268043A072182
:102690003345280000000000E50D0000150E000085
:1026A0001815AF19FF1815AE19FF00000001140A24
:1026B0006464323200127A00000428961008000088
:1026C000800040001815A115C819FF1815AE15D5C2
:1026D000168015A8163F15D316001540158D161433
:1026E0001520160015A115C815DA1612158116CF7A
:1026F00015D916F115DB1640152E15A415A619FFD0
:102700001815A015C019FF506F776572204D6574BC
:102710006572205265762E203100352D6469676917
:10272000742055534220747970652D430043414C09
:102730004942524154494E47006D757874726F6E2C
:102740006963732E6E6C0000F8B5C046F8BC08BC17
:102750009E467047B5000000F8B5C046F8BC08BCFE
:082760009E4670478D00000049
:10276800010000000727000023608000246080002B
:1027780001000000392700001A2700002D2700005B
:04000003000000F108
:00000001FF
